:100000000C9465020C94A9020C94A9020C94A90208
:100010000C94A9020C94A9020C94A9020C94A902B4
:100020000C94A9020C94A9020C94C50B0C94970C87
:100030000C94A9020C94A9020C94A9020C94A90294
:100040000C94A9020C9422210C94A9020C94A902EC
:100050000C94A9020C94C41A0C94A9020C94A90241
:100060000C94A9020C94A9020C94A9020C94A90264
:100070000C94A9020C94A9020C94A9020C94A90254
:100080000C94A9020C94A9020C94A9020C94A90244
:100090000C94A9020C94A9020C94A9020C94A90234
:1000A0000C94A9020C94A9020C94A902FC0C1E0D3C
:1000B000090E1E0D090E600D830D090ED80DEB0DF6
:1000C000D810D81006110611481184118413841316
:1000D0009C118413931293125E138413841372136E
:1000E0000000F0A12E004C002A00E1003581000044
:1000F0001E00140004001D7134004D001F001A0082
:1001000016001B00E1042A0020000800070006007A
:1001100050002C0021001500090019004F004A0072
:10012000220017000A000500000065745000015409
:100130000000007F0000E3004F0001540000007742
:100140000000E20023001C000B00110000002971D8
:10015000240018000D00100052004B0025000C0078
:100160000E00360051002800260012000F00370054
:100170002F002B00270013003382387130004E000F
:100180002D0031003478E500C100000001000100BD
:1001900001000100010000003A001E0220022202BC
:1001A000010001003B001F022102230201000100A7
:1001B0003C002F0226022F00010001003D0030020A
:1001C00027023000010001003E00310235003502F7
:1001D000000001000100010000000100000001001A
:1001E0000100010000000100000001003F0052007A
:1001F00051002402000001004000240021001E00E4
:10020000010001004100250022001F00370001000D
:1002100042002600230020002700010043002502A1
:100220002E0231002E0001004400450001000100B3
:1002300001000000010001000100010001000000B8
:1002400001000100010001000100010001000100A6
:10025000F2000100010001000100F000F1000100C6
:10026000F400010001000100F3000100F5000100AD
:100270000100010001000100000001000100010077
:100280000000010000000100010001000000010069
:100290000000010001000100010001000000010058
:1002A0000100010001000100A9000100010001009E
:1002B0000100AC00AA00B600010001000100AB0083
:1002C000A80001000100010001000100010001007F
:1002D00001000100AE00010001000000160345000E
:1002E000720067006F0044006F0078002000450036
:1002F0005A00000016034500720067006F004400BA
:100300006F007800200045005A0000000403090433
:1003100009026D00040100A0FA09040000010301B4
:100320000100092111010001223F00070581030896
:10033000000A090401000103010200092111010062
:1003400001224D000705820308000A09040200018A
:100350000300000009211101000122360007058376
:100360000308000A09040300010300000009211129
:100370000100012239000705840310000112011059
:100380000100000008EDFE07130100010200010555
:10039000010906A101050719E029E71500250195C6
:1003A0000875018102050819012905950575019156
:1003B000029501750391010507190029771500259C
:1003C00001957875018102C005010980A1018502AE
:1003D00016010026B7001A01002AB7007510950112
:1003E0008100C0050C0901A1018503160100269CAE
:1003F000021A01002A9C02751095018100C00501B6
:100400000902A1010901A100050919012905150029
:10041000250195057501810295017503810105018D
:10042000093009311581257F950275088106093843
:100430001581257F950175088106050C0A3802157E
:1004400081257F950175088106C0C005010906A1B7
:1004500001050719E029E7150025019508750181B7
:100460000295017508810105081901290595057591
:100470000191029501750391010507190029FF15E6
:100480000025FF950675088100C0000000000000EF
:100490000000000000010204060A0F17202C3A4A4F
:1004A0005D71879DB3C7DAE9F5FCFFFCF5E9DAC7B2
:1004B000B39D87715D4A3A2C20170F0A060402018A
:1004C0000000000000000000000011241FBECFEF5C
:1004D000DAE0DEBFCDBF04B603FE24C08091EE019A
:1004E0009091EF01A091F001B091F1018730904B14
:1004F000A740B04BB9F41092EE011092EF011092A8
:10050000F0011092F10114BE84B7877F84BF88E1A7
:100510000FB6F89480936000109260000FBEE0E088
:10052000FFE3099511E0A0E0B1E0E8ECF5E402C0DA
:1005300005900D92A433B107D9F711E0A4E3B1E01F
:1005400001C01D92AE3EB107E1F70E940B090C9469
:10055000E2220C94000061110BC0FC01828188230F
:1005600021F085EE0E946C0F03C085EE0E943410CE
:1005700080E090E0089508956091B1017091B2011A
:100580008091B3019091B4010E94F01956985E9841
:1005900025982D9826982E9827982F98813019F015
:1005A000823021F00895259A2D9A0895269A2E9A40
:1005B00008958CEB92E0892B11F00E94BC0280E040
:1005C00090E0089556985E9825982D9826982E9834
:1005D00027982F988FEF90E0909389008093880060
:1005E00090938B0080938A0090938D0080938C0071
:1005F000259A2D9A2FEF80E792E02150804090407D
:10060000E1F700C00000269A2E9A2FEF80E792E0D3
:10061000215080409040E1F700C00000279A2F9AB7
:100620002FEF80E792E0215080409040E1F700C03A
:10063000000025982D982FEF80E792E02150804010
:100640009040E1F700C0000026982E982FEF80E739
:1006500092E0215080409040E1F700C000002798D0
:100660002F9856985E9825982D9826982E9827981A
:100670002F98089589EA8093800089E08093810013
:1006800024982C983F988AB18F748AB96E98479AAB
:100690008BB1806B8BB9769A0E94E2028BEB92E071
:1006A000892B11F00E94BB0280E090E0089580E267
:1006B000809300018091340181110EC00E94A60335
:1006C00081E0809334012FEF83ED90E3215080404F
:1006D0009040E1F700C0000080E40E94AC038093EA
:1006E000000181112EC00E94D60380930001811168
:1006F00028C00E94D60380930001811122C08FE39D
:100700000E94D6038093000181111BC00E94CE037A
:1007100080E40E94AC0380930001811112C08CE040
:100720000E94D6038093000181110BC00E94D60362
:1007300080930001811105C08FE30E94D60380934E
:1007400000010E94CE038091000108951092B9002B
:100750008AE08093B800089594EA9093BC00909149
:10076000BC0097FFFCCF9091B900987F983021F0A2
:10077000903111F081E008958093BB0084E880936C
:10078000BC008091BC0087FFFCCF8091B900887FBE
:10079000883111F0803471F780E0089584E9809306
:1007A000BC008091BC0084FDFCCF08958093BB0009
:1007B00084E88093BC008091BC0087FFFCCF9091BF
:1007C000B900987F81E0983209F480E0089584E8C8
:1007D0008093BC008091BC0087FFFCCF8091BB0060
:1007E000089580910001811115C080E40E94AC033E
:1007F0008093000181110CC082E10E94D603809396
:100800000001811105C08FEF0E94D6038093000183
:100810000E94CE0384B1807F84B985B1807F85B981
:100820008AB1837F8AB98BB1837F8BB93E98469812
:1008300008950E945703809300010E94F10380B342
:100840008C7080BB81B3836F81BBE4E4F1E0A6E3ED
:10085000B1E011921D9281E0E235F807D1F78AE309
:1008600093E0892B11F00C943A030895BF92CF9234
:10087000DF92EF92FF920F931F93CF93DF938091BC
:100880000001882379F0809135018F5F80933501D5
:10089000811108C00E94570380930001811102C09A
:1008A0000E94E20206E311E0C0E0D0E0DD24D39430
:1008B00082E0C82EEE24E394F12CC73000F580913D
:1008C0000001811162C080E40E94AC0380930001AA
:1008D000811112C082E10E94D60380930001811130
:1008E0000BC0C7010C2E01C0880F0A94EAF780954F
:1008F0000E94D603809300010E94CE0346C0CA30F6
:10090000A1F028F4C83059F0C93061F005C0CC30EE
:1009100089F070F0CD3089F0209A289810C0219A83
:1009200029980DC0229A2A980AC0239A2B9807C0AA
:10093000529A01C0539A5B9802C03E9A4698E0EAE8
:10094000EA95F1F78FB1799960C092E081708D25B9
:10095000892B7C9B02C090E001C094E0892B7D9B99
:1009600002C090E001C098E0892B7E9B02C090E01D
:1009700001C090E1892B9FB19095991F9927991FEC
:100980009295990F907E892B0FC080910001811163
:1009900051C080E40E94AC03809300018823B9F128
:1009A000B12C0E94CE038B2DF8019081981719F07D
:1009B0008083C09201010E94F10321960F5F1F4FB7
:1009C000CE30D10509F079CF809101018823B1F0B3
:1009D000815080930101882339F08FE99FE00197CE
:1009E000F1F700C000000AC0A4E4B1E0E6E3F1E0E2
:1009F00081918D9391E0E434F907D1F789ED92E08C
:100A0000892BD1F00E94D90217C090E09FCF83E1DB
:100A10000E94D603809300018111C2CF81E40E941D
:100A2000AC03809300018111BBCF0E94E703B82E75
:100A3000B094B7CF80E0B8CF81E0DF91CF911F9124
:100A40000F91FF90EF90DF90CF90BF900895E82F27
:100A5000F0E0EC5BFE4F8081089508958B3B91059B
:100A600078F4883A910540F5853A9105D0F48430C0
:100A7000910508F0B1C08130910509F4ADC06BC09B
:100A8000803E910508F467C0883E910508F4A4C033
:100A90009C01205F31092031310508F05CC0906570
:100AA0000895853A910509F459C0863A910509F4EB
:100AB00058C083E890E40895883A910509F454C039
:100AC000893A910509F453C08A3A910509F452C054
:100AD0008B3A910509F451C08C3A910509F450C044
:100AE0008D3A910509F44FC0803B910509F44EC041
:100AF0008E3A910509F44DC08F3A910509F44CC026
:100B0000813B910509F44BC0823B910509F44AC031
:100B1000833B910509F449C0843B910509F448C021
:100B2000853B910509F447C0863B910509F446C011
:100B3000873B910509F445C0883B910509F444C001
:100B4000893B910509F443C08A3B910509F042C0F5
:100B50008AE296E4089580E090E0089581E890E4C8
:100B6000089582E890E4089582EE94E4089589EE71
:100B700094E408958AEE94E4089585EB94E408954E
:100B800086EB94E4089587EB94E408958CEC94E468
:100B900008958DEC94E4089583E895E408958AE837
:100BA00095E4089582E995E4089584E995E408952B
:100BB00081E296E4089583E296E4089584E296E45F
:100BC000089585E296E4089586E296E4089587E222
:100BD00096E4089580E094E40895089596E0799F5E
:100BE000F001112494E5899FE00DF11D1124E60F19
:100BF000F11DEE0FFF1FEC51FF4F85919491089569
:100C0000880F991F805A9040FC0185919491089516
:100C1000880F991F80529F4FFC01859194910895F0
:100C200026E0729FF001112444E5849FE00DF11D40
:100C30001124E60FF11DEE0FFF1FEC51FF4F259120
:100C40003491C9019A9581159F4110F4C901089505
:100C5000C90190528115904128F4C9019F700E94EA
:100C600008060895C90190538115904120F4C901E7
:100C70009927906C0895211580E5380769F40E9442
:100C8000A5139FEF24E34CE0915020404040E1F752
:100C900000C000000C94E91A213080E5380731F4D7
:100CA0008091CC0181608093CC010895C901905559
:100CB0008115904108F050C0832F99278F70992794
:100CC00081309105D9F4A9014370552702C0880FDE
:100CD000991F4A95E2F79C68A90164E0440F551FEB
:100CE0006A95E1F744275370842B952B73E0220F0C
:100CF000331F7A95E1F7207633271DC082309105A6
:100D000029F4922F8827816F906A08958330910586
:100D1000A9F4A9014370552781E090E002C0880F33
:100D2000991F4A95E2F79C6843E0220F331F4A95CA
:100D3000E1F7207E3770822B932B08950497F1F40E
:100D4000A9014370552781E090E002C0880F991FE8
:100D50004A95E2F79A68E8CFC9019057811590410A
:100D600020F4C9019F7090620895C90190588115BF
:100D7000904120F4C9019F70906A0895203E31058A
:100D8000E0F4203C310558F52133310509F470C0F9
:100D900048F42932310509F464C02A32310509F4D6
:100DA0006EC074C029333105F1F022383105D9F015
:100DB0002533310509F44EC069C0233E310589F160
:100DC00038F4203E3105C1F0223E3105E1F05EC02D
:100DD000263E310569F1273E3105A9F157C0C90109
:100DE0000E94000608958091DF0180FD02C081FF0E
:100DF0004DC080EE90E04BC08091DF0180FFF9CFC5
:100E000089E390E044C08091DF0182FF0EC08091B1
:100E1000DF0184FF03C080E090E039C083EE90E002
:100E200036C08091DF0182FFF2CF82EE90E02FC0CA
:100E30008091DF0183FF0BC08091DF0184FDEBCF48
:100E400087EE90E024C08091DF0183FFF5CF86EE2E
:100E500090E01DC08091DF0185FF07C089E290E02E
:100E600016C08091DF0185FFF9CF85E390E00FC0C8
:100E70008091DF0186FF07C08AE290E008C0809180
:100E8000DF0186FFF9CF81E390E001C0C9010E9434
:100E90002E0508950895809162010895CF93DF9300
:100EA00000D01F92CDB7DEB72091E501243019F5AF
:100EB00023E029839B838A832093E9008FEF90911D
:100EC000E800815095FD06C095ED9A95F1F7000078
:100ED0008111F5CF8091E80085FF0DC040E050E022
:100EE00063E070E0CE0101960E94B8098091E800AD
:100EF0008E778093E8000F900F900F90DF91CF9145
:100F00000895CF93DF9300D01F92CDB7DEB7209125
:100F1000E501243021F522E029839B838A8383E045
:100F20008093E9008FEF9091E800815095FD06C015
:100F300095ED9A95F1F700008111F5CF8091E800C9
:100F400085FF0DC040E050E063E070E0CE01019607
:100F50000E94B8098091E8008E778093E8000F9096
:100F60000F900F90DF91CF9108952091E5012430EB
:100F7000F1F422E02093E9002FEF3091E8002150B6
:100F800035FD06C035ED3A95F1F700002111F5CF9A
:100F90002091E80025FF0BC040E050E065E070E0E4
:100FA0000E94B8098091E8008E778093E800089548
:100FB000CF93DF93EC018091E501843009F046C0C6
:100FC00090910C019923D9F090910D019923B9F0DA
:100FD0008093E9008FEF9091E800815095FD06C065
:100FE00095E19A95F1F700008111F5CF8091E80025
:100FF00085FF2CC040E050E060E170E017C081E068
:101000008093E9008FEF9091E800815095FD06C034
:1010100095ED9A95F1F700008111F5CF8091E800E8
:1010200085FF14C040E050E068E070E0CE010E940F
:10103000B8098091E8008E778093E80080E1FE0196
:10104000A2E5B1E001900D928A95E1F7DF91CF9191
:1010500008958091E401811109C00E944A0B0E9409
:10106000A70B8091E20084608093E20008951092C3
:10107000E401089508950C940F210E94801A0E94A3
:1010800015210E94440E0C944A0742E061EC81E075
:101090000E94C40A42E061EC82E00E94C40A42E07D
:1010A00061EC83E00E94C40A42E161EC84E00C94AC
:1010B000C40A8091E701833009F455C030F48130CF
:1010C00071F0823009F48EC008958A3009F47AC034
:1010D0008B3009F460C0893009F09CC020C0809139
:1010E000E601813A09F096C08091E800877F8093FD
:1010F000E8008091EA019091EB01892B21F060E0FA
:1011000080E090E003C060E182E591E070E00E9441
:10111000010A8091E8008B778093E8000895809120
:10112000E601813209F076C08091EA019091EB01ED
:10113000009719F0039709F06DC08091E800877F50
:101140008093E8008091E80082FD05C08091E50170
:101150008111F8CF5FC08091F1008093620180918E
:10116000E8008B7753C08091E601813A09F052C0C4
:101170008091EA019091EB01892B09F04BC080919D
:10118000E800877F8093E8008091E80080FFFCCF33
:1011900080910C0136C08091E6018132D9F58091B1
:1011A000EA019091EB01892BA9F58091E800877FF6
:1011B0008093E8000E94F90A8091E80180930C0175
:1011C0000C94A5138091E601813221F58091E8000D
:1011D000877F8093E8000E94F90A8091E90180935B
:1011E000630108958091E601813AA1F48091E800BD
:1011F000877F8093E8008091E80080FFFCCF80919A
:1012000063018093F1008091E8008E778093E8007D
:101210000C94F90A089584B7877F84BF88E10FB6DC
:10122000F89480936000109260000FBE90E080E818
:101230000FB6F89480936100909361000FBE0E94F6
:10124000930E0E944A0B0E94A70B8091E2008460DB
:101250008093E20078940E94220E0E94950E82E014
:1012600091E00E943F0E0E94FD208091E5018530B3
:1012700069F40E94431A8091E3018823B1F30E942C
:101280006B1A882391F30E94A209EFCF0E949B0E54
:10129000ECCF292F332723303105A9F06CF421300E
:1012A000310509F442C02230310509F043C08DE612
:1012B00090E020E133E042C021323105C9F0223212
:1012C000310519F137C099278130910541F08230FD
:1012D000910541F0892B71F5ECE0F3E005C0E4EFF6
:1012E000F2E002C0ECEDF2E0849190E09F0126C0B4
:1012F000643000F5E62FF0E0EE0FFF1FEE5DFE4FCD
:101300002081318189E090E019C0643098F4E62FA3
:10131000F0E0DF01AA0FBB1FA65EBE4F2D913C91EE
:10132000EA5EFE4F808190E009C082E190E02DE707
:1013300033E004C080E090E020E030E0FA01318347
:101340002083089580E189BD82E189BD09B400FE52
:10135000FDCF8091D8008F7D8093D8008091E000F0
:1013600082608093E0008091E00081FDFCCF0895D1
:10137000CF92DF92EF92FF920F931F93CF93DF9361
:101380007C018B01EA010E941A0B811131C0209768
:1013900031F088819981081B190BE80EF91EC12CC8
:1013A000D12C0115110519F18091E80085FD14C0BB
:1013B0008091E8008E778093E800209741F0888143
:1013C00099818C0D9D1D9983888385E011C00E94B1
:1013D0001A0B882331F30CC0F70181917F018093B0
:1013E000F10001501109FFEFCF1ADF0ADACF80E0D8
:1013F000DF91CF911F910F91FF90EF90DF90CF90F1
:1014000008952091EC013091ED012617370748F03F
:101410006115710539F42091E8002E772093E800DA
:1014200001C0B901FC0120E061157105B9F180919D
:10143000E501882309F440C0853009F43FC080915C
:10144000E80083FD3DC08091E80082FF06C08091E6
:10145000E80082FF26C080E008958091E80080FFC8
:10146000E3CF2091F3008091F20090E0922B611580
:10147000710551F08830910538F421912093F100E5
:10148000615071090196F3CF21E0089709F020E03F
:101490008091E8008E778093E800C6CF2111C7CFF6
:1014A000D6CF8091E501882339F0853039F08091DD
:1014B000E80083FFCCCF04C082E0089583E0089564
:1014C00081E008952091EC013091ED012617370756
:1014D00048F06115710539F42091E8002E772093CA
:1014E000E80001C0B901FC0120E061157105C1F1FE
:1014F0008091E501882309F441C0853009F440C09A
:101500008091E80083FD3EC08091E80082FF06C024
:101510008091E80082FF27C080E008958091E80074
:1015200080FFE3CF2091F3008091F20090E0922BB6
:101530006115710559F08830910540F4249120938C
:10154000F1003196615071090196F2CF21E00897C0
:1015500009F020E08091E8008E778093E800C5CF05
:101560002111C6CFD5CF8091E501882339F0853090
:1015700039F08091E80083FFCBCF04C082E008956A
:1015800083E0089581E00895982F973058F590935F
:10159000E900981739F07091EC002091ED0050911E
:1015A000F00003C0242F762F50E021FF19C03091A6
:1015B000EB003E7F3093EB003091ED003D7F3093A8
:1015C000ED003091EB0031603093EB007093EC0054
:1015D0002093ED005093F0002091EE0027FF07C00C
:1015E0009F5FD3CF8F708093E90081E0089580E002
:1015F00008958091E60187FD05C08091E80080FF95
:101600000EC012C08091E80082FD05C08091E50106
:101610008111F8CF08958091E8008B7708C0809100
:10162000E5018111EACF08958091E8008E778093DB
:10163000E80008958091E4009091E50045E620914E
:10164000EC0020FF21C02091E80020FD21C0209166
:10165000E501222389F0253089F02091EB0025FD5A
:101660000FC02091E4003091E5002817390739F3C5
:10167000415041F0C901E3CF82E0089583E008952D
:1016800081E0089584E008952091E80022FFDFCFF3
:1016900080E008950E94B80B0E94C00BE0EEF0E0DD
:1016A000808181608083E8EDF0E080818F778083A6
:1016B00019BCA7EDB0E08C918E7F8C9380818F7EDA
:1016C00080831092E40108950F931F93CF93DF93CB
:1016D0000E94B80B0E94C00BC8EDD0E088818F77C4
:1016E000888388818068888388818F7D888319BCFE
:1016F0001092E5011092E1011092E3011092E201D3
:1017000000EE10E0F80180818B7F8083888181600A
:10171000888342E060E080E00E94C40AE1EEF0E0ED
:1017200080818E7F8083E2EEF0E080818160808323
:10173000808188608083F80180818E7F80838881AA
:1017400080618883DF91CF911F910F910895E8ED1B
:10175000F0E080818F7E8083E7EDF0E08081816022
:10176000808384E082BF81E08093E4010C94640B69
:10177000E8EDF0E080818E7F80831092E200089592
:101780001092DA001092E10008951F920F920FB6A6
:101790000F9211242F933F934F935F936F937F93F7
:1017A0008F939F93AF93BF93EF93FF938091E1004B
:1017B00082FF0BC08091E20082FF07C08091E100B0
:1017C0008B7F8093E1000E94210E8091DA0080FFE0
:1017D0001FC08091D80080FF1BC08091DA008E7FEF
:1017E0008093DA008091D90080FF0DC080E189BD2F
:1017F00082E189BD09B400FEFDCF81E08093E5015F
:101800000E94290805C019BC1092E5010E94370802
:101810008091E10080FF19C08091E20080FF15C037
:101820008091E2008E7F8093E2008091E2008061EF
:101830008093E2008091D80080628093D80019BC28
:1018400085E08093E5010E943B088091E10084FFE0
:1018500030C08091E20084FF2CC080E189BD82E12C
:1018600089BD09B400FEFDCF8091D8008F7D8093A3
:10187000D8008091E1008F7E8093E1008091E200AA
:101880008F7E8093E2008091E20081608093E2008D
:101890008091E101882311F084E007C08091E3008A
:1018A00087FF02C083E001C081E08093E5010E94D0
:1018B0003D088091E10083FF29C08091E20083FF11
:1018C00025C08091E100877F8093E10082E08093D2
:1018D000E5011092E1018091E1008E7F8093E100AB
:1018E0008091E2008E7F8093E2008091E20080612F
:1018F0008093E20042E060E080E00E94C40A8091B0
:10190000F00088608093F0000E943A08FF91EF9108
:10191000BF91AF919F918F917F916F915F914F9107
:101920003F912F910F900FBE0F901F9018951F920F
:101930000F920FB60F9211242F933F934F935F9303
:101940006F937F938F939F93AF93BF93CF93EF93B7
:10195000FF93C091E900CF708091EC001092E900F4
:101960008091F000877F8093F00078940E94D30CE0
:101970001092E9008091F00088608093F000C0939D
:10198000E900FF91EF91CF91BF91AF919F918F911E
:101990007F916F915F914F913F912F910F900FBE6B
:1019A0000F901F9018951F93CF93DF93CDB7DEB79D
:1019B000AA970FB6F894DEBF0FBECDBFE6EEF1E0FA
:1019C0008091F100819321E0EE3EF207C9F70E9479
:1019D00059088091E80083FF1CC12091E6013091F5
:1019E000E701832F90E08A30910508F012C1FC01D5
:1019F000EA5AFF4F0C949722203881F0223809F0E0
:101A000008C18091EA018F708093E9008091EB001A
:101A100085FB882780F91092E90006C08091E201D9
:101A20009091E301911182609091E800977F9093EB
:101A3000E8008093F1001092F100C5C0822F8D7FE5
:101A400009F0E7C0222319F0223061F0E2C0809152
:101A5000E801813009F0DDC0333009F080E0809387
:101A6000E30128C08091E801811124C02091EA019E
:101A70002F7009F4CEC02093E9008091EB0080FF25
:101A800019C08091EB00333011F4806211C0806185
:101A90008093EB0081E090E0022E01C0880F0A9451
:101AA000EAF78093EA001092EA008091EB008860E8
:101AB0008093EB001092E9008091E800877F86C058
:101AC0002111A7C01091E8011F778091E300807871
:101AD000812B8093E3008091E800877F8093E8006A
:101AE0000E94F90A8091E80080FFFCCF8091E3001A
:101AF00080688093E300112311F083E001C082E04D
:101B00008093E50186C02058223008F082C0809181
:101B1000E8019091E9018C3D23E0920779F583E09B
:101B20008A838AE289834FB7F894DE01139620E016
:101B30003EE051E2E32FF0E050935700E49120FFA4
:101B400003C0E295EF703F5FEF708E2F90E0EA30B8
:101B500010F0C79601C0C0968D939D932F5F2431DE
:101B600049F74FBF8091E800877F8093E8006AE2E1
:101B700070E0CE0101960E94010A14C0AE014F5FD1
:101B80005F4F6091EA010E944909009709F441C042
:101B90002091E800277F2093E800BC0189819A8189
:101BA0000E94620A8091E8008B778093E80031C040
:101BB000203879F58091E800877F8093E800809154
:101BC000E1018093F1008091E8008E778093E80036
:101BD0000E94F90A1EC021111CC09091E8019230A8
:101BE000C0F48091E800877F8093E8009093E10142
:101BF0000E94F90A8091E101811104C08091E30003
:101C000087FF02C084E001C081E08093E5010E946B
:101C100045088091E80083FF0AC08091E800877F33
:101C20008093E8008091EB0080628093EB00AA969D
:101C30000FB6F894DEBF0FBECDBFDF91CF911F91DD
:101C400008950895CF938091E5018823B1F08091A4
:101C5000E9008F709091EC0090FF02C090E801C005
:101C600090E0C92FC82B1092E9008091E80083FD15
:101C70000E94D30CCF70C093E900CF910895909348
:101C80006901809368010895E0916801F09169010C
:101C9000309721F00190F081E02D099480E00895C3
:101CA000E0916801F0916901309721F00280F381A1
:101CB000E02D09940895E0916801F0916901309751
:101CC00021F00480F581E02D0994089520916601AA
:101CD000309167018217930771F0909367018093A9
:101CE0006601E0916801F0916901309721F006806A
:101CF000F781E02D099408952091640130916501E8
:101D00008217930771F09093650180936401E091CD
:101D10006801F0916901309721F00084F185E02D90
:101D20000994089508950C94920E0E94861A0E94B8
:101D300019040C944C1BCF92DF92EF92FF920F93F9
:101D40001F93CF93DF93CDB7DEB72B970FB6F894E1
:101D5000DEBF0FBECDBF0E9436043BE6E32E31E06E
:101D6000F32E00E010E0C02E802F0E942705F7011F
:101D7000D1907F01D826B1F40F5F1F4F0E301105AF
:101D800091F78FEF89838A831B820E948F1A81606B
:101D9000782F9D838C8349815A816B818D810E942C
:101DA0003E0F41C09091CC0191FF04C08B870E94EF
:101DB0002D058B8520E030E04D2D50E0922FBA01AB
:101DC000022E02C0759567950A94E2F760FF25C060
:101DD0002E83CF82EE24E394F12C02C0EE0CFF1C84
:101DE0009A95E2F790E08E219F2121E0892B09F45A
:101DF00020E028870E948F1A8160782F9A87898730
:101E00004E815F8168858A850E943E0FF801E55901
:101E1000FE4F80818E25808306C02F5F3F4F263086
:101E2000310561F6A9CF0E94301E10916A010E940F
:101E3000440E1817A1F00E94440E80936A012B965D
:101E40000FB6F894DEBF0FBECDBFDF91CF911F91CB
:101E50000F91FF90EF90DF90CF900C944A072B9654
:101E60000FB6F894DEBF0FBECDBFDF91CF911F91AB
:101E70000F91FF90EF90DF90CF900895CF93DF9375
:101E8000CDB7DEB72B970FB6F894DEBF0FBECDBF30
:101E90004F83588769877A878B87DE01119686E0A2
:101EA000FD0111928A95E9F785E0FE0137960190D0
:101EB0000D928A95E1F749815A816B817C818D81F0
:101EC0009E810E9471162B960FB6F894DEBF0FBE4E
:101ED000CDBFDF91CF910895CF93C82F882309F408
:101EE000C1C0823859F40E94440E81FDBBC089E311
:101EF0000E9410190E94CA1989E30CC0833879F432
:101F00000E94440E80FDAEC083E50E9410190E941D
:101F1000CA1983E50E945019CF910C94CA198438CC
:101F200059F40E94440E82FD9DC087E40E9410195E
:101F30000E94CA1987E4EECF8CEF8C0F813A48F4E7
:101F40008C2F0E94652081118DC08C2F0E9410194A
:101F5000E3CF80E28C0F883048F4C77081E001C085
:101F6000880FCA95EAF70E949119D6CF8BE58C0F9E
:101F7000833078F4C53A29F0C63A31F482E890E02B
:101F800005C081E890E002C083E890E0CF910C9416
:101F9000660E88E58C0F833108F064C0C83A39F1C9
:101FA000C93A41F1CA3A49F1CB3A51F1CC3A59F127
:101FB000CD3A61F1C03B69F1CE3A71F1CF3A79F196
:101FC000C13B81F1C23B89F1C33B91F1C43B99F123
:101FD000C53BA1F1C63BA9F1C73BB1F1C83BB9F183
:101FE000C93BC1F1CA3BC9F58AE292E038C082EE32
:101FF00090E035C089EE90E032C08AEE90E02FC0CC
:1020000085EB90E02CC086EB90E029C087EB90E058
:1020100026C08CEC90E023C08DEC90E020C083E8DB
:1020200091E01DC08AE891E01AC082E991E017C0F2
:1020300084E991E014C081E292E011C083E292E071
:102040000EC084E292E00BC085E292E008C086E216
:1020500092E005C087E292E002C080E090E0CF917C
:102060000C947C0ECF910895882309F44BC08238DC
:1020700059F40E94440E81FF45C089E30E94101963
:102080000E94CA1989E30CC0833871F40E94440E7F
:1020900080FF38C083E50E9410190E94CA1983E5A9
:1020A0000E9450190C94CA19843859F40E94440EA5
:1020B00082FF28C087E40E9410190E94CA1987E491
:1020C000EFCF9CEF980F913A58F390E2980F983029
:1020D00050F4877091E001C0990F8A95EAF7892F33
:1020E0000E949719DFCF9BE5980F933020F480E092
:1020F00090E00C94660E885A833120F480E090E0E2
:102100000C947C0E0895882321F00E9491190C9460
:10211000CA190895882321F00E9497190C94CA19AE
:102120000895CF92DF92EF92FF920F931F93CF9378
:10213000DF93CDB7DEB728970FB6F894DEBF0FBE9A
:10214000CDBF8C0185E0F801DE01119601900D9262
:102150008A95E1F7F80140813181F280258122954D
:102160002F7083819481892B31F03F3F31F481E0DE
:102170004F3F19F403C081E001C080E080FDC4C27C
:1021800049833A8389819A812F830E94CE189E8346
:1021900088870E94CD180E94A0174E81E42FE295F7
:1021A000EF70F0E0E05AFF4F2F8168850C94972282
:1021B000842F807F142F1F70882311F01295107FB9
:1021C000FF2059F0112309F454C2812F68870E941F
:1021D000A1190E94CA1968854CC2862F0E9434102A
:1021E000112309F491C2812F0E94A71928960FB6D6
:1021F000F894DEBF0FBECDBFDF91CF911F910F913D
:10220000FF90EF90DF90CF900C94CA19342F307F5D
:10221000842F8F70303211F08295807F662319F001
:10222000613019F12BC0FF20B1F0222309F493C1D2
:10223000213009F090C128960FB6F894DEBF0FBE8A
:10224000CDBFDF91CF911F910F91FF90EF90DF9065
:10225000CF900C94B119222319F0213009F454C203
:102260008E830E94B4198E8189C1FF2021F0223013
:1022700008F04AC270C1211147C280C1FF2021F07D
:10228000222309F468C1F5C1222309F477C105C2EC
:10229000242F26952695237030E02115310521F055
:1022A00021303105C9F030C2FF2021F0862F942F54
:1022B000937002C080E090E028960FB6F894DEBFDD
:1022C0000FBECDBFDF91CF911F910F91FF90EF9087
:1022D000DF90CF900C94660EFF2021F0862F942F74
:1022E000937002C080E090E028960FB6F894DEBFAD
:1022F0000FBECDBFDF91CF911F910F91FF90EF9057
:10230000DF90CF900C947C0E862FFF2019F00E9456
:10231000381D02C00E94A01D28960FB6F894DEBF9B
:102320000FBECDBFDF91CF911F910F91FF90EF9026
:10233000DF90CF900C94251E842F837009F076C017
:10234000F110E2C1262F229526952770220F220F29
:10235000862F8F70C82ED12CE12CF12C022E04C0B8
:10236000CC0CDD1CEE1CFF1C0A94D2F764FF10C0DD
:102370006FE070E080E090E004C0660F771F881F78
:10238000991F2A95D2F7609570958095909503C016
:1023900060E070E0CB01242F269526952370422F14
:1023A00050E042305105D1F04330510559F16C29CC
:1023B0007D298E299F294130510541F128960FB67C
:1023C000F894DEBF0FBECDBFDF91CF911F910F916B
:1023D000FF90EF90DF90CF900C94C5176C297D296A
:1023E0008E299F2928960FB6F894DEBF0FBECDBF69
:1023F000DF91CF911F910F91FF90EF90DF90CF90E1
:102400000C94DF170E94C517C701B60128960FB6B6
:10241000F894DEBF0FBECDBFDF91CF911F910F911A
:10242000FF90EF90DF90CF900C94AB17FF2019F046
:10243000842F817001C08695882309F465C1262FF9
:10244000229526952770220F220F862F8F70C82E77
:10245000D12CE12CF12C022E04C0CC0CDD1CEE1C86
:10246000FF1C0A94D2F764FF10C06FE070E080E0B8
:1024700090E004C0660F771F881F991F2A95D2F736
:10248000609570958095909503C060E070E0CB01F9
:10249000242F269526952370422F50E04230510577
:1024A000D1F04330510559F16C297D298E299F299E
:1024B0004130510541F128960FB6F894DEBF0FBEAA
:1024C000CDBFDF91CF911F910F91FF90EF90DF90E3
:1024D000CF900C9499186C297D298E299F292896D4
:1024E0000FB6F894DEBF0FBECDBFDF91CF911F9125
:1024F0000F91FF90EF90DF90CF900C94B3180E9453
:102500009918C701B60128960FB6F894DEBF0FBE22
:10251000CDBFDF91CF911F910F91FF90EF90DF9092
:10252000CF900C947F18603FC9F118F4603E50F4CE
:102530009BC0623F09F460C008F44AC0633F09F4DD
:102540006FC092C0162F1F70842F8F71FF2099F0DB
:102550000E941818812F28960FB6F894DEBF0FBE80
:10256000CDBFDF91CF911F910F91FF90EF90DF9042
:10257000CF900C9483100E943918812F28960FB6A3
:10258000F894DEBF0FBECDBFDF91CF911F910F91A9
:10259000FF90EF90DF90CF900C948A10FF20A1F075
:1025A0002111B2C0842F8F7128960FB6F894DEBF28
:1025B0000FBECDBFDF91CF911F910F91FF90EF9094
:1025C000DF90CF900C945E18223008F09DC0EACFC7
:1025D000FF20A1F0842F8F7128960FB6F894DEBFEC
:1025E0000FBECDBFDF91CF911F910F91FF90EF9064
:1025F000DF90CF900C941818FF2061F3842F8F7117
:1026000028960FB6F894DEBF0FBECDBFDF91CF91F5
:102610001F910F91FF90EF90DF90CF900C9439189D
:10262000FF2091F0842F8F7128960FB6F894DEBFAB
:102630000FBECDBFDF91CF911F910F91FF90EF9013
:10264000DF90CF900C94031828960FB6F894DEBF55
:102650000FBECDBFDF91CF911F910F91FF90EF90F3
:10266000DF90CF900C94F917FF20A1F0222309F4FA
:10267000B1CF862F28960FB6F894DEBF0FBECDBF20
:10268000DF91CF911F910F91FF90EF90DF90CF904E
:102690000C946C0F222309F4B1CF862F28960FB625
:1026A000F894DEBF0FBECDBFDF91CF911F910F9188
:1026B000FF90EF90DF90CF900C9434104F70C801D2
:1026C0000E94AB0228960FB6F894DEBF0FBECDBFB6
:1026D000DF91CF911F910F91FF90EF90DF90CF90FE
:1026E0000C941E174F70C80128960FB6F894DEBFE1
:1026F0000FBECDBFDF91CF911F910F91FF90EF9053
:10270000DF90CF900C94ED0528960FB6F894DEBFBD
:102710000FBECDBFDF91CF911F910F91FF90EF9032
:10272000DF90CF9008950E94AE190E9483190E94F5
:10273000CA190E94D11E0E94251E80E090E00E94CE
:10274000660E80E090E00C947C0E0E949E190C9422
:1027500093130E94CE18292F22952F7030E02C3031
:1027600031054CF42A3031056CF422503109223005
:10277000310590F407C02C30310551F02F30310570
:1027800039F00AC0803E10F0803F31F481E00895B6
:1027900093FB882780F9089580E00895CF93DF9315
:1027A00000D000D01F92CDB7DEB70F900F900F90E2
:1027B0000F900F90DF91CF910895CF93DF9300D0CA
:1027C00000D000D0CDB7DEB726960FB6F894DEBFA6
:1027D0000FBECDBFDF91CF9108951F93CF93DF93AD
:1027E000C091790116E080917A01C81799F0D0E084
:1027F0001C9FF0011D9FF00D1124E558FE4F4081F4
:10280000518162817381848195810E94DD132196BB
:10281000C770E9CFDF91CF911F9108954091AB012F
:102820005091AC016091AD017091AE018091AF010A
:102830009091B0010C94DD13CF938091B0018295FB
:102840008F7009F05FC08091AD01882309F45AC0F0
:1028500020917901A0917A016091AB017091AC0156
:102860008091AE019091AF0131E06F3F09F030E00F
:10287000B32FC6E02A1709F445C0009721F07F3F27
:1028800021F44B2F03C041E001C040E030E040FDA7
:1028900035C0C29FF001C39FF00D1124E558FE4FD3
:1028A000418174132BC04081641328C042814111BF
:1028B00025C0438154814817590710F441505109EC
:1028C000481B590B483C5105C8F48091B0018F70EA
:1028D00080618093B00186E0829FF001839FF00DBC
:1028E0001124E058FE4F80818F70806180838BEAD5
:1028F00091E00E949110CF910C94ED132F5F3F4F08
:102900002770B8CFCF910895CF92DF92EF92FF92C8
:102910000F931F93CF93DF93CDB7DEB762970FB6B8
:10292000F894DEBF0FBECDBF8C0185E0F801DE015B
:102930001D9601900D928A95E1F7D8014C91119660
:102940005C91119712966C9112971396ED90FC90F2
:1029500014977091AB01E091AC012091AE013091E0
:10296000AF012115310531F0EF3F31F481E07F3FB8
:1029700019F403C081E001C080E0B82FB170CB2E04
:1029800080FD6CC1D090AD01DD2009F4F5C0F0915F
:10299000B001E216F30638F0C701821B930B883CA6
:1029A000910548F09BC0209530952E0D3F1D283C89
:1029B000310508F093C08F2F807F09F052C0E513D6
:1029C00014C0741312C0D62E61110FC0FF70F061D5
:1029D000F093B0010E940E148BEA91E00E949110D6
:1029E0008091B001F80185836CC1EF2831F05F3F21
:1029F00031F481E04F3F19F403C081E001C080E071
:102A000080FD03C081E0862701C080E0F82FF170CF
:102A1000FF2E80FF1CC08091790120917A0136E061
:102A2000821709F428C190E0389FF001399FF00D1A
:102A30001124E558FE4F7181571306C0708147136A
:102A400003C07281671303C001968770E9CFD62E49
:102A5000662309F436C18091B00181608093B00192
:102A600053C0E51308C0741306C0611104C0D80137
:102A70001596FC93AEC04D875E878D859E856A8BCB
:102A80000E94A9136A89882329F1D62E662311F1A1
:102A90002091B001822F82958F7090E002970CF404
:102AA00060C08091AB019091AC0198878F831986AB
:102AB000FB86EA862C87CE01079651C0E51731F1D7
:102AC0004D875E878D859E856A8B0E94A9136A89D2
:102AD00081112EC0C8010E949110A4C08F2F807F49
:102AE00069F77E2DF98AE88A89890E94CE138BEADC
:102AF00091E00E949110EBEAF1E086E0DF011D9287
:102B00008A95E9F70E940E14D12CDBC07413D8CF3C
:102B10006111D6CFD8011596FC93C8010E9491107F
:102B2000EBEAF1E086E0DF011D928A95E9F7C9C082
:102B3000D62E662379F22091B001822F82958F7074
:102B400090E0029774F08091AB019091AC019A8370
:102B500089831B82FD82EC822E83CE0101960E9426
:102B6000911086E0F801ABEAB1E001900D928A95F0
:102B7000E1F70E941C146FC0E216F30628F0C701AB
:102B8000821B930B9C0104C0209530952E0D3F1D98
:102B9000283C310508F052C0D62E662309F49ACF9E
:102BA000E5132CC074132AC08091B00180FD1DC0B4
:102BB000982F92959F70C9F0D80115968C93159710
:102BC0009F3039F09F5F9295907F8F70892B15967B
:102BD0008C93C8010E94911086E0F801ABEAB1E045
:102BE00001900D928A95E1F736C086E0F801ABEAD4
:102BF000B1E001900D928A95E1F763C04D875E8741
:102C00008D859E850E94A913882379F086E0F801BE
:102C1000ABEAB1E001900D928A95E1F70E941C1495
:102C20000E940E14DD24D3944CC08091B0018160C9
:102C30008093B001C8010E94911043C07E2DF98A93
:102C4000E88A89890E94CE13EBEAF1E086E0DF0191
:102C50001D928A95E9F70E940E1433C0662309F489
:102C600039CF4D875E878D859E850E94A913882365
:102C700009F430CFCBCF4D875E878D859E850E942E
:102C8000CE18292F22952F7030E0223031052CF4F8
:102C90009F7041F0811106C00CC0243031052CF426
:102CA0009F7049F4805E883020F0C8010E94911026
:102CB000CF2CDC2C06C0D80115969C91907F91F703
:102CC000F8CF8D2D62960FB6F894DEBF0FBECDBF44
:102CD000DF91CF911F910F91FF90EF90DF90CF90F8
:102CE00008951F93CF93DF93CDB7DEB72C970FB620
:102CF000F894DEBF0FBECDBF4F83588769877A87B0
:102D00008B879C87CE0107960E9484148823C1F08C
:102D10002F8138858A859B85892B31F03F3F11F0C3
:102D200080E003C02F3FE1F781E0811147C04F8170
:102D3000588569857A858B859C850E94DD133EC008
:102D400086E0FE013796DE01119601900D928A957C
:102D5000E1F7FF81E8854A855B854115510531F032
:102D6000EF3F31F481E0FF3F19F403C081E001C07F
:102D700080E080FD23C020917A0130E0C9010196F6
:102D8000877099276091790170E086179707F1F1B4
:102D9000F983EA835D834C8396E0929FD001939FF1
:102DA000B00D1124A558BE4FFE01319601900D9231
:102DB0009A95E1F780937A010E94ED1316E08091D5
:102DC000790190917A01891779F1189FC001112436
:102DD00085589E4F0E948414882331F1E091790137
:102DE0001E9FF0011124E558FE4F40815181628100
:102DF0007381848195810E94DD138091790190E037
:102E000001968770992780937901D9CF0E94A513E5
:102E100010927A0110927901EBEAF1E086E0DF018D
:102E20001D928A95E9F7CACF2C960FB6F894DEBFAB
:102E30000FBECDBFDF91CF911F910895EF92FF920A
:102E40000F931F93CF93DF939C01009709F471C0F8
:102E5000F12CEE24E394E9012196F9018491843761
:102E600040F4843008F056C0813081F0823021F186
:102E700060C0853709F449C0C0F19CE7980F9037CE
:102E800008F057C08F770E94341046C089010E5F4A
:102E90001F4FFE01849190E2980F983050F4877094
:102EA000FE2D01C0FF0F8A95EAF78F2F0E94A1190E
:102EB00015C00E946C0F14C089010E5F1F4FFE01E8
:102EC000849190E2980F983068F48770FE2D01C0CD
:102ED000FF0F8A95EAF78F2F0E94A7190E94CA193F
:102EE000E8011AC00E943410FBCF2E5F3F4FFE0155
:102EF000C491CC2341F08FE99FE00197F1F700C026
:102F00000000C150F6CFE90107C0FE01F490E901CD
:102F1000229602C00E946C0F8F2D882341F0EFE9AA
:102F2000FFE03197F1F700C000008150F6CF9E011D
:102F300092CFDF91CF911F910F91FF90EF90089565
:102F400008956093B5017093B6018093B701909393
:102F5000B8010C9493130F931F930091B501109136
:102F6000B6012091B7013091B801062B172B282B01
:102F7000392B0093B5011093B6012093B70130931C
:102F8000B8011F910F910C9493130F931F9300910D
:102F9000B5011091B6012091B7013091B801062317
:102FA0001723282339230093B5011093B6012093EA
:102FB000B7013093B8011F910F910C9493130F93A5
:102FC0001F930091B5011091B6012091B701309186
:102FD000B80106271727282739270093B501109332
:102FE000B6012093B7013093B8011F910F910C9453
:102FF00093131092B1011092B2011092B30110928A
:10300000B4010C94931341E050E060E070E004C020
:10301000440F551F661F771F8A95D2F74093B10161
:103020005093B2016093B3017093B4010C94931365
:1030300041E050E060E070E004C0440F551F661F9F
:10304000771F8A95D2F78091B1019091B201A0913A
:10305000B301B091B401842B952BA62BB72B809391
:10306000B1019093B201A093B301B093B4010C9459
:10307000931341E050E060E070E004C0440F551F3E
:10308000661F771F8A95D2F7409550956095709589
:103090008091B1019091B201A091B301B091B401BE
:1030A00084239523A623B7238093B1019093B20183
:1030B000A093B301B093B4010C94931341E050E09A
:1030C00060E070E004C0440F551F661F771F8A95AB
:1030D000D2F78091B1019091B201A091B301B0916A
:1030E000B40184279527A627B7278093B101909331
:1030F000B201A093B301B093B4010C9493130F9356
:103100001F930091B1011091B2012091B301309150
:10311000B401062B172B282B392B0093B1011093E8
:10312000B2012093B3013093B4011F910F910C941D
:1031300093130F931F930091B1011091B20120914D
:10314000B3013091B40106231723282339230093B8
:10315000B1011093B2012093B3013093B4011F91D8
:103160000F910C9493130F931F930091B101109141
:10317000B2012091B3013091B40106271727282707
:1031800039270093B1011093B2012093B30130931A
:10319000B4011F910F910C9493130895CF92DF9275
:1031A000EF92FF920F931F93CF93DF93EC01C090A8
:1031B000B501D090B601E090B701F090B8018091D0
:1031C000B1019091B201A091B301B091B401C82AAC
:1031D000D92AEA2AFB2A0FE110E0B701A601002E46
:1031E00004C076956795579547950A94D2F740FFA6
:1031F00007C0BE01802F0E9410068130910539F46E
:103200000150110950F7BE0180E00E941006DF91C5
:10321000CF911F910F91FF90EF90DF90CF90089585
:1032200090910C019923D9F090910D019923B9F057
:10323000982F9695969596959F3088F5E0910E017A
:10324000F0910F01E90FF11D877021E030E001C01E
:10325000220F8A95EAF78181822B8183089540911C
:103260000E0150910F0120E030E09FEFFA01E20FD4
:10327000F31F6281681799F09F3F19F4611101C033
:10328000922F2F5F3F4F2E30310581F79F3F39F04E
:10329000FA01E90FF11D97FDFA95828308950895CB
:1032A00090910C019923E1F090910D019923C1F0C7
:1032B000982F9695969596959F3020F5E0910E0162
:1032C000F0910F01E90FF11D877021E030E001C09E
:1032D000220F8A95EAF7209581812823218308957A
:1032E00040910E0150910F0120E030E0FA01E20F11
:1032F000F31F9281981301C012822F5F3F4F2E302F
:103300003105A1F7089581E090E0E0910E01F09180
:103310000F01E80FF91F1082019680319105A9F77E
:1033200008959091CB01982B9093CB0108958095AF
:103330009091CB0198239093CB0108951092CB01EB
:1033400008959091CA01982B9093CA010895809591
:103350009091CA0198239093CA0108951092CA01CE
:1033600008958093B90108951092B901089540918C
:103370000E0150910F0120E030E080E0FA01E20FF1
:10338000F31F918191118F5F2F5F3F4F2F303105D8
:10339000A9F70895E0910E01F0910F018091CB0102
:1033A0008083E0910E01F0910F0180819091CA011C
:1033B000892B80839091B901992361F0E0910E01EE
:1033C000F0910F018081892B80830E94B7198111B0
:1033D0001092B90180910E0190910F010C94500E42
:1033E000CF92DF92EF92FF920F931F936C01EE2426
:1033F000FF24C114D104E104F10421F46B017C0128
:1034000080E001C080E133272F2D1E2D0D2D0115E9
:1034100011052105310519F0885F680179019701CF
:103420008601A4E03695279517950795AA95D1F7BB
:10343000011511052105310519F08C5F680179012D
:1034400097018601F2E03695279517950795FA952D
:10345000D1F7011511052105310519F08E5F6801BD
:103460007901B701A6017695679557954795452B44
:10347000462B472B09F08F5F1F910F91FF90EF9024
:10348000DF90CF9008958091E501843009F110928A
:10349000CD0120E488E190E00FB6F894A8958093E0
:1034A00060000FBE2093600083B7817F846083BF7C
:1034B00083B7816083BF7894889583B78E7F83BFFD
:1034C00088E10FB6F89480936000109260000FBE00
:1034D000089508950895CF930E94691A0E943604B2
:1034E0000E946A1AC0E08C2F0E942705811105C036
:1034F000CF5FCE30C1F780E001C081E0CF91089569
:103500000E94A5130E94440E0C944A0782E084BDD9
:1035100093E095BD9AEF97BD80936E0008952FB705
:10352000F8948091CE019091CF01A091D001B091FB
:10353000D1012FBF0895CF92DF92EF92FF920F93A8
:103540001F932FB7F8944091CE015091CF01609115
:10355000D0017091D1012FBF6A017B01EE24FF24BD
:103560008C0120E030E0C016D106E206F30610F42C
:1035700041505109481B590BCA011F910F91FF90EF
:10358000EF90DF90CF9008951F920F920FB60F9299
:1035900011248F939F93AF93BF938091CE0190910D
:1035A000CF01A091D001B091D1010196A11DB11D13
:1035B0008093CE019093CF01A093D001B093D1011D
:1035C000BF91AF919F918F910F900FBE0F901F9061
:1035D00018950E944A0BF8942FEF87EA91E6215044
:1035E00080409040E1F700C0000087E090EBDC01F4
:1035F0008093EE019093EF01A093F001B093F1015D
:103600002CE088E190E00FB6F894A89580936000D4
:103610000FBE20936000FFCFEF92FF920F931F9396
:10362000CF93DF93E82EF12C8F2D0E942705C0E069
:10363000D0E0082F10E098010C2E02C03595279598
:103640000A94E2F720FD05C02196C630D10599F70E
:1036500009C06C2F7F2D80E00E94EE05E812F4CFA8
:1036600081E005C0F3948EE0F812DECF80E0DF91B8
:10367000CF911F910F91FF90EF900895CF93C82F96
:103680008CE20E940C1B882321F08C2FCF910C948C
:103690000C1B80E0CF910895CF930E94911C811163
:1036A00002C00E94771CC5E6C15049F00E94360452
:1036B0008FE39CE90197F1F700C00000F5CF89E2A4
:1036C0000E943E1B811111C18AE20E943E1B8111A2
:1036D0000E94771C85E00E943E1B81110E94E91A1E
:1036E0000E949C1C8093CC0187E00E943E1B882393
:1036F00099F18BE10E943E1B882351F09091CC01FF
:1037000091FB882780F921E0822780FB91F922C074
:103710008EE00E943E1B882351F09091CC0192FBD9
:10372000882780F921E0822780FB92F913C080E18D
:103730000E943E1B9091CC01882341F093FB882787
:1037400080F921E0822780FB93F904C0892F8095BE
:1037500080FB90F99093CC018091CC010E94A01C39
:103760000E94AE1C8093DF0180EE0E943E1B8823E6
:1037700041F08091DF01982F909590FB80F9809324
:10378000DF0189E30E943E1B882359F09091DF01FD
:1037900091FB882780F921E0822780FB91F99093A3
:1037A000DF0182EE0E943E1B882359F09091DF01D9
:1037B00092FB882780F921E0822780FB92F9909381
:1037C000DF0186EE0E943E1B882359F09091DF01B5
:1037D00093FB882780F921E0822780FB93F990935F
:1037E000DF0183EE0E943E1B882359F09091DF0198
:1037F00094FB882780F921E0822780FB94F990933D
:10380000DF0185E30E943E1B882359F09091DF0180
:1038100095FB882780F921E0822780FB95F990931A
:10382000DF0181E30E943E1B882359F09091DF0164
:1038300096FB882780F921E0822780FB96F99093F8
:10384000DF0181E10E943E1B882359F09091DF0146
:1038500097FB882780F921E0822780FB97F99093D6
:10386000DF018091DF010E94B21C8091DF0187FBA4
:10387000882780F980930D0187E20E943E1BC82FA4
:103880008EE10E943E1B8111C2608FE10E943E1BAF
:103890008111C46080E20E943E1B8111C86081E2F8
:1038A0000E943E1B8111C06182E20E943E1B811179
:1038B000C06283E20E943E1B8111C06484E20E94C8
:1038C0003E1B882311F0C06802C0CC2329F08C2F46
:1038D0000E94A91C6C2F03C00E94A51C682F70E0D9
:1038E00080E090E0CF910C94A117CF9108956DEEF8
:1038F0007EEF80E090E00E94CD2260E082E090E0E8
:103900000E94BF2260E083E090E00E94BF2260E05E
:1039100084E090E00E94BF2260E085E090E00C949B
:10392000BF2280E090E00E94B92221E08D3E9E4FB0
:1039300009F020E0822F089582E090E00C94B122FB
:10394000682F82E090E00C94BF2283E090E00C941A
:10395000B122682F83E090E00C94BF2284E090E0D5
:103960000C94B122682F84E090E00C94BF228091E7
:10397000D40180FF0BC06091130185E0689FB00106
:10398000112475956795759567952AC081FF09C0C3
:103990006091130185E0689FB001112475956795CA
:1039A0001FC082FF07C06091130185E0689FB001CE
:1039B000112416C04091D5014423C9F06091120131
:1039C000461788F72091130185E0289F9001112464
:1039D000429FC001439F900D112470E00E948322FA
:1039E0006038710540F46115710539F002C065E079
:1039F00070E0862F08958FE7089581E00895809103
:103A0000D40180FF08C06091110170E07595679541
:103A10007595679521C081FF06C06091110170E026
:103A20007595679519C082FF04C06091110170E01F
:103A300010C08091D5018823C1F0609110018617D4
:103A4000A0F790911101989FC001112470E00E948D
:103A500083226038710528F46115710521F0862FE5
:103A600008958FE7089581E0089561E070E0F4CF54
:103A7000803F21F40E94B71C819504C0813F29F446
:103A80000E94B71C8093D8010895823F21F40E94C0
:103A9000B71C819504C0833F29F40E94B71C809312
:103AA000D7010895893F19F40E94FF1C05C08A3F81
:103AB00031F40E94FF1C81958093D90108958B3FBA
:103AC00021F40E94FF1C819504C08C3F29F40E94C0
:103AD000FF1C8093DA010895843F21F48091D60180
:103AE000816017C0853F21F48091D601826011C0AA
:103AF000863F21F48091D60184600BC0873F21F47A
:103B00008091D601886005C0883F31F48091D6014C
:103B100080618093D60108958D3F21F48091D40176
:103B200081600BC08E3F21F48091D401826005C07A
:103B30008F3F29F48091D40184608093D40108954B
:103B4000803F39F48091D80187FF6CC01092D80172
:103B500069C0813F29F48091D8011816BCF362C076
:103B60009091D701823F29F497FF5CC01092D70152
:103B700059C0833F19F41916CCF354C0893F41F45E
:103B80008091D90118160CF04DC01092D9014AC08D
:103B90008A3F29F48091D90187FF44C0F6CF8B3F3B
:103BA00039F48091DA0187FF3DC01092DA013AC002
:103BB0008C3F29F48091DA011816BCF333C0843F9E
:103BC00021F48091D6018E7F17C0853F21F480912A
:103BD000D6018D7F11C0863F21F48091D6018B7F65
:103BE0000BC0873F21F48091D601877F05C0883FB5
:103BF00031F48091D6018F7E8093D60113C08D3F22
:103C000021F48091D4018E7F0BC08E3F21F48091EE
:103C1000D4018D7F05C08F3F29F48091D4018B7F23
:103C20008093D4018091D70181110EC08091D80179
:103C300081110AC08091D901811106C08091DA01F9
:103C4000811102C01092D501089586ED91E00E9485
:103C50005B0E0E948F1A9093D3018093D201089536
:103C60001F93CF93DF938091D2019091D3010E9453
:103C70009B1A4091D501442321F02091140130E09A
:103C800006C0209115015AE0259F9001112482174A
:103C9000930708F482C08091D7011091D801D09188
:103CA000D901C091DA01811107C0111105C0D111EC
:103CB00003C0CC2309F471C04F3F19F04F5F40930C
:103CC000D501181624F40E94B71C8093D701809167
:103CD000D70187FF05C00E94B71C81958093D7014B
:103CE000111624F40E94B71C8093D8018091D8014A
:103CF00087FF05C00E94B71C81958093D801609111
:103D0000D701662339F11091D801112319F17727D2
:103D100067FD7095872F972F0E94942123E333E34B
:103D200043E35FE30E94F8210E9461216093D70181
:103D3000612F772767FD7095872F972F0E94942119
:103D400023E333E343E35FE30E94F8210E94612110
:103D50006093D8011D1624F40E94FF1C8093D901A2
:103D60008091D90187FF05C00E94FF1C8195809337
:103D7000D9011C1624F40E94FF1C8093DA01809163
:103D8000DA0187FF05C00E94FF1C81958093DA014C
:103D9000DF91CF911F910C94251EDF91CF911F9140
:103DA0000895E6EDF1E085E0DF011D928A95E9F7DF
:103DB0001092D5011092D4010895833081F128F436
:103DC000813059F08230D1F00895853009F449C02E
:103DD000B8F1863009F456C0089520911501862F58
:103DE00090E0820F911D8F3F910520F4620F609348
:103DF000150108958FEF8093150108952091140106
:103E0000862F90E0820F911D8F3F910520F4620F65
:103E10006093140108958FEF809314010895209109
:103E20001301862F90E0820F911D8F3F910520F4A2
:103E3000620F6093130108958FEF8093130108952B
:103E400020911201862F90E0820F911D8F3F9105E6
:103E500020F4620F6093120108958FEF8093120196
:103E6000089520911101862F90E0820F911D8F3FC0
:103E7000910520F4620F6093110108958FEF8093F4
:103E80001101089520911001862F90E0820F911D5D
:103E90008F3F910520F4620F6093100108958FEF1A
:103EA000809310010895833011F128F4813049F096
:103EB000823091F00895853081F120F18630C1F192
:103EC000089580911501681720F4861B80931501D1
:103ED000089510921501089580911401681720F437
:103EE000861B809314010895109214010895809107
:103EF0001301681720F4861B809313010895109214
:103F00001301089580911201681720F4861B809395
:103F100012010895109212010895809111016817FD
:103F200020F4861B809311010895109211010895C9
:103F300080911001681720F4861B8093100108956A
:103F40001092100108958D3109F442C020F58E3091
:103F500009F479C070F4873009F45EC020F486302B
:103F600009F442C033C08830D1F18B3009F4A7C0C6
:103F70002DC0863109F4A3C038F4803109F46DC036
:103F8000813109F47BC022C0893109F498C08B319A
:103F900009F44FC01BC0853309F479C048F4873257
:103FA00009F475C008F478C0893209F470C00EC0F5
:103FB000833438F48A3308F071C0883309F47FC041
:103FC00005C0833409F463C08834C1F080E00895EB
:103FD0000E941B210E94440E0E944A0770C00E944A
:103FE0009C1C0E94AE1C6BC08091CC01817F8E7F97
:103FF0008093CC0181E08093DC0108950E94A51399
:104000002FEF83ED90E3215080409040E1F700C016
:1040100000000E94E91A53C09091CC01892F817051
:1040200090FF03C0917F9E7F26C091609093CC014A
:1040300046C09091CC0191FB882780F921E082272E
:1040400080FB91F913C09091CC0192FB882780F9F5
:1040500021E0822780FB92F909C09091CC0193FB6B
:10406000882780F921E0822780FB93F99093CC0187
:10407000882329F191609093CC0108950E94A513A3
:1040800080910D0191E0892780930D0118C061E0B6
:1040900070E080E090E00FC023EE01C027EC280F15
:1040A00061E070E080E090E004C0660F771F881F39
:1040B000991F2A95D2F70E94A1170E94A51381E0AB
:1040C000089580E0089580E00895CF93C82F8091EF
:1040D000DC01813079F018F08230D1F184C0A091F8
:1040E0000E01B0910F018C91813169F0823209F09B
:1040F0007CC009C0A0910E01B0910F018C9181315B
:1041000011F0823249F48C2F0E94612081111DC070
:104110008C2F0E94A31F1AC08C2F0E946320811134
:1041200014C0C43179F048F4CB3079F0C03109F0D3
:1041300060C082E08093DC0108C0C93219F0C83346
:1041400021F057C01092DC0154C081E0817053C04F
:10415000C93289F118F5C43171F1A8F4C73009F0FA
:1041600046C08AE08093150194E19093140193E096
:10417000909313018093120188E08093110188E2EB
:104180008093100134C0CE51C63088F5EC2FF0E09A
:10419000E65DFE4F80818093DB0129C0CE34E9F0DB
:1041A00020F4CB3421F56AE013C0C13579F0C23573
:1041B000F1F461E00DC08091DB01882319F01092C9
:1041C000DB0115C081E08093DC0115C061E006C011
:1041D0008091DB010E94DD1E0AC06AE08091DB0154
:1041E0000E94531F04C01092DC0180E004C081E0F3
:1041F00002C080E0ABCFCF910895E1E8F0E080818C
:10420000886080838081816080838FB7F89493E099
:104210009093890090ED909388008FBF0895EFE60A
:10422000F0E08081826080830895EFE6F0E0808195
:104230008D7F80830895EFE6F0E0808192E089270A
:10424000808308951F920F920FB60F9211242F931F
:104250003F934F935F936F937F938F939F93AF930E
:10426000BF93EF93FF938091DD019091DE01019662
:104270009093DE018093DD01811103C082E00E94F2
:104280004A07E091DE01E695E695F0E0E657FB4F40
:10429000E4918091DD018E1303C080E00E944A0703
:1042A000FF91EF91BF91AF919F918F917F916F910E
:1042B0005F914F913F912F910F900FBE0F901F90E4
:1042C000189504D06894B1118DC0089570D088F00D
:1042D0009F5790F0B92F9927B751A0F0D1F0660FF2
:1042E000771F881F991F1AF0BA95C9F712C0B1300D
:1042F00081F077D0B1E0089574C0672F782F8827B8
:10430000B85F39F0B93FCCF3869577956795B3954B
:10431000D9F73EF490958095709561957F4F8F4FBA
:104320009F4F0895E89409C097FB3EF490958095BF
:10433000709561957F4F8F4F9F4F9923A9F0F92F6B
:1043400096E9BB279395F695879577956795B795E9
:10435000F111F8CFFAF4BB0F11F460FF1BC06F5FCF
:104360007F4F8F4F9F4F16C0882311F096E911C0E1
:10437000772321F09EE8872F762F05C0662371F002
:1043800096E8862F70E060E02AF09A95660F771F16
:10439000881FDAF7880F9695879597F9089557FD46
:1043A0009058440F551F59F05F3F71F04795880FA3
:1043B00097FB991F61F09F3F79F08795089512163A
:1043C00013061406551FF2CF4695F1DF08C01616E6
:1043D00017061806991FF1CF869571056105089497
:1043E0000895E894BB2766277727CB0197F90895AE
:1043F0000BD078C069D028F06ED018F0952309F062
:104400005AC05FC01124EECFCADFA0F3959FD1F34D
:10441000950F50E0551F629FF001729FBB27F00D72
:10442000B11D639FAA27F00DB11DAA1F649F6627C7
:10443000B00DA11D661F829F2227B00DA11D621F16
:10444000739FB00DA11D621F839FA00D611D221FD0
:10445000749F3327A00D611D231F849F600D211DB4
:10446000822F762F6A2F11249F5750408AF0E1F057
:1044700088234AF0EE0FFF1FBB1F661F771F881FA0
:1044800091505040A9F79E3F510570F014C0AACF3B
:104490005F3FECF3983EDCF3869577956795B7958B
:1044A000F795E7959F5FC1F7FE2B880F911D9695B5
:1044B000879597F9089597F99F6780E870E060E025
:1044C00008959FEF80EC089500240A9416161706AD
:1044D00018060906089500240A94121613061406F5
:1044E00005060895092E0394000C11F4882352F058
:1044F000BB0F40F4BF2B11F460FF04C06F5F7F4F10
:104500008F4F9F4F089597FB072E16F4009407D006
:1045100077FD09D00E949D2207FC05D03EF49095BE
:1045200081959F4F0895709561957F4F0895EE0F87
:10453000FF1F0590F491E02D0994AA1BBB1B51E1CC
:1045400007C0AA1FBB1FA617B70710F0A61BB70B03
:10455000881F991F5A95A9F780959095BC01CD01A8
:104560000895F999FECF92BD81BDF89A992780B53B
:104570000895A8E1B0E042E050E00C94D422262F48
:10458000F999FECF1FBA92BD81BD20BD0FB6F89438
:10459000FA9AF99A0FBE019608950E94BF22272F1A
:1045A0000C94C022DC01CB01FC01F999FECF06C0BE
:1045B000F2BDE1BDF89A319600B40D9241505040E1
:0845C000B8F70895F894FFCF4D
:1045C80020024B07D807B50781074E070101BA013A
:1045D80028080A03140A3F4D36394B04FE03C80362
:1045E8008F0322033B0354036D03010203040506F2
:0445F80007080900A7
:00000001FF
